:1000000003C003C003C003C003C003C003C003C0D8
:10008000BEC3E8C3E7C3E6C3E5C3E4C3E3C3E2C357
:10009000E1C3E0C3DFC3DEC3DDC3DCC3DBC317C022
:1000A00016C04CC014C009021200010100803209C0
:1000B000040000000000000012011001FF00000811
:1000C000D01653070A01000000010403090411249B
:1000D0001FBECFE5D2E0CDBFDEBF00EB0F9307E040
:1000E0000F9310E0A0E6B0E0EAEDFFE102C005905A
:1000F0000D92A636B107D9F720E0A6E6B0E001C020
:100100001D92AB39B207E1F7ECC1A82FB92F80E0FF
:1001100090E041E050EA609530E009C02D918227DF
:100120009795879510F084279527305EC8F36F5F09
:10013000A8F30895EADF8D939D930895CF93CFB7E9
:10014000CF93C0915F02C03B21F4C0915E02C730E3
:1001500021F0CF91CFBFCF91A1CFCC27C395B39B37
:10016000E9F7B39B0BC0B39B09C0B39B07C0B39B1C
:1001700005C0B39B03C0B39B01C0D3C00F92DF93F4
:10018000C0917E00DD27CB57DF4F012EB39B03C00C
:10019000DF910F90E6CF2F930F931F934F932FEF85
:1001A0004F6F06B303FB20F95F933F9350E03BE0B2
:1001B00065C016B30126502953FDC89556B30127D3
:1001C00003FB25F92F7306B3B1F05027102713FB5B
:1001D00026F906B22230F0F000C016B3012703FB67
:1001E00027F90126502906B22430E8F54F77206818
:1001F00016B30000F6CF50274F7D206206B2102FB5
:10020000000000C006B300265029102713FB26F972
:1002100006B2E2CF4F7B06B3206400C0DACF0126DE
:100220005029187106B269F14E7F2160012F16B373
:1002300028C0002650294D7F06B22260102F29C009
:10024000012650294B7F06B22460012F2DC016B322
:1002500001265029477F2860000006B22EC04F7E3D
:1002600006B3206130C0422706B3499300265029C7
:10027000102706B24FEF13FB20F9297F16B379F24E
:10028000187159F10126502906B2012703FB21F903
:10029000237F06B371F2002650293150D0F006B208
:1002A000102713FB22F9277E16B351F2012650299D
:1002B000012703FB06B223F92F7C49F2000006B3A5
:1002C000102713FB24F90026502906B22F7939F2A2
:1002D00070CF10E21ABF002717C03B503195C31BE7
:1002E000D04010E21ABF0881033CF9F00B34E9F06A
:1002F00020917C001981110F1213EDCF093651F1B5
:100300000D3211F0013E39F7009383003F915F9168
:100310004F911F910F912F91DF910F90CAB7C5FD9B
:100320001DCFCF91CFBFCF9118952091830022236D
:1003300069F310918100112321F5343022F13093BB
:10034000810020937D0010917E003BE0311B3093B3
:100350007E0019C00091810001309CF40AE53091C3
:10036000600034FD11C000936000C1E7D0E010C010
:10037000052710E000C021C0052710E0C89508BB84
:1003800014C03AE501C032ED032EC0E0D0E032E007
:1003900017B31861C39A08B317BB58E120E84FEFB1
:1003A00020FF052708BB279517951C3F28F700005D
:1003B0004552B0F720FF0527279508BB17951C3F2E
:1003C000B8F629913A9561F7077E10918200110FD6
:1003D00008BBC250D04011F010937C0010E21ABF4D
:1003E000086017B3177E402F477E54E05A95F1F707
:1003F00008BB17BB48BB8ACFF8942FEFB0E8A0E446
:100400004AE0B1BF000081EE9CE0B399FECFB39B00
:10041000FECF0197B399FDCF97FF03C0BA1B81951B
:1004200001C0BA0FA69529F4281710F031B7282F6C
:10043000A1E0415031F731BF000078940895F8945D
:10044000E0916A00F0916B00329785E0809357004D
:10045000E89578940895E0916A00F0916B003097E8
:1004600029F490936D0080936C0007C0E430F1058F
:1004700039F490936F0080936E008FE39CEC1CC066
:10048000EC3728E1F20739F480916C0090916D000F
:100490008E539C4F11C0EE3728E1F20739F480915A
:1004A0006E0090916F008D539C4F06C0EA3728E193
:1004B000F20711F481B790E02FB7F894309721F448
:1004C00031E130935700E89531E00C01309357004B
:1004D000E89511243296F0936B00E0936A002FBFE9
:1004E000089514BE88E10FB6F89481BD11BC0FBE0B
:1004F000C198BB9A88E893E1ECE9F1E03197F1F714
:100500000197D1F7BB98AC9A8BB780628BBF789478
:1005100000918100035007FDBAC080917E00CCE0BD
:10052000D0E0C81BD109CB57DF4F80917D008D32C1
:1005300009F08EC0083009F0A8C083EC80937100E8
:100540008AE580936000109269002881922F90764E
:100550008981992319F110926700811108C082E600
:1005600090E09093800080937F0014E067C081301A
:1005700051F48C819D8190936B0080936A0027FDDC
:1005800058C01FEF57C090916800823011F49160FD
:1005900001C094609093680010E050C09A8110925E
:1005A0007A00811106C010927B008AE790E012E089
:1005B0003BC0853019F4909382002CC0863009F539
:1005C0008B81813019F48AE998E104C0823041F4CA
:1005D00088E898E19093800080937F0012E10DC03D
:1005E000833051F4911108C08CEA98E19093800017
:1005F00080937F0014E001C010E080E480936900E4
:100600001DC0883059F0893019F49093840002C0DD
:100610008A3039F08AE790E010E006C084E890E084
:1006200002C08AE790E011E09093800080937F0001
:1006300005C01E8180E88093690007C08F81811109
:1006400004C08E81811708F4182F109361001DC01B
:100650008091690087FF19C080916A0090916B00BA
:100660008038984128F080916A008F7339F00DC06E
:1006700089919991F0DE025079F7F5CF8091680069
:1006800082608093680010926100109281008091D6
:10069000600084FF43C0809161008F3F09F43EC039
:1006A000082F893008F008E0801B8093610080915A
:1006B000710098E8892780937100002319F1E09177
:1006C0007F00F09180008091690086FF0BC0A2E757
:1006D000B0E084918D93319682E790E0800F8A1389
:1006E000F8CF0CC0CF01A2E7B0E0FC012191CF010F
:1006F0002D9322E730E0200F2A13F7CFF0938000EC
:10070000E0937F00602F82E790E014DD0C5F0C30F7
:1007100019F08FEF809361000093600084E196B33D
:10072000987131F48150D9F71092820010927C00B8
:1007300001E0811100E080917000801739F0011113
:1007400003C01092670058DE009370008CE991E0BE
:100750000197F1F70091680000FF17C0F894E0E8F6
:10076000F8E1E054F10983E080935700E895309771
:10077000C1F710926B0010926A0088E0F82E8FEF9C
:100780009FEF69DEFA94D9F75ADE01FF05C08AE3CC
:1007900090E20197F1F753DE02FF13C0B99882E2AD
:1007A00091EA0197F1F7F894BB9A1BBE15BA109223
:1007B0005F02EAE7F8E1E4918E2F81508E3FC0F0AE
:1007C00019C010926800809167008D7011F0B9987F
:1007D00001C0B99A8091660090916700019690934C
:1007E00067008093660080369A4E08F491CED6CF8B
:1007F000E1BF000052CC22CF5AFF187A4008000017
:1008000000000000000000000000000000000000E8
:1008100000000000000000000000000000001124A3
:100820001FBECFE5D2E0DEBFCDBF10E0A0E6B0E056
:10083000EAEBFAE002C005900D92A236B107D9F7B3
:1008400010E0A2E6B0E001C01D92A236B107E1F7C8
:100850001CD131C115CC05C0EDE1F0E13197F1F7C4
:1008600001970097C9F70895AC01407C80E090E0C3
:10087000FC01E40FF51F25913491FC01EE7FE60F9A
:10088000F71F2083318302968034910589F70895FC
:10089000FC01E07C83E080935700E89507B600FCFC
:1008A000FDCF0895CF93DF93EC01AB01DB0120E096
:1008B00030E0FE01E41BF50BEA0FFB1F8D919D91CB
:1008C00061E00C0160935700E89511242F5F3F4FC2
:1008D0002032310571F785E0FE0180935700E895DD
:1008E00007B600FCFDCFDF91CF910895CF93DF9342
:1008F000CDB7DEB7C054D0400FB6F894DEBF0FBE00
:10090000CDBF809160009091610096958795815050
:100910009044FE0131969E012F5B3F4F819391934E
:10092000E217F307D9F780E090E0B2DF80E090E0D3
:10093000BE016F5F7F4FB6DFC05CDF4F0FB6F8942C
:10094000DEBF0FBECDBFDF91CF9108950F931F93F0
:10095000CF93DF93CDB7DEB7C054D0400FB6F89435
:10096000DEBF0FBECDBF00E010E040C080E090E0F1
:10097000F801E256FF4FE80FF91F9C0135952795C6
:1009800047E0EE3FF40770F0F901EE0FFF1F21E0A2
:1009900030E02C0F3D1FE20FF31F2FEF3FEF3183AD
:1009A00020830DC045915491F901EE0FFF1F21E006
:1009B00030E02C0F3D1FE20FF31F4083518302965E
:1009C00080349105A9F68091600090916100800FBC
:1009D000911F5EDF8091600090916100800F911FF8
:1009E000BE016F5F7F4F5EDF005C1F4F37E0003856
:1009F000130709F0BBCFC05CDF4F0FB6F894DEBF22
:100A00000FBECDBFDF91CF911F910F910895CF936E
:100A1000DF93CDB7DEB7C054D0400FB6F894DEBF39
:100A20000FBECDBF80E090E0BE016F5F7F4F1CDF47
:100A30008FEF9FEF9A83898380E090E029DF80E049
:100A400090E0BE016F5F7F4F2DDFC05CDF4F0FB6C0
:100A5000F894DEBF0FBECDBFDF91CF910895CF9345
:100A600087B3836087BBC198CAEF81E090E0F3DE73
:100A7000C19A81E090E0EFDEC198C150B1F7CF910B
:100A80000895E0E0F0E00995089588B318BA87B3B7
:100A90008FEF87BB8AEF90E0DEDE87B317BA8AEF6D
:100AA00090E0D9DEF894B3DF51DF20DFD8DFE9DF53
:0A0AB00080E090E00895F894FFCF75
:020ABA008018A2
:040000030000008079
:00000001FF
